:100000004CC066C065C064C063C062C061C060C0EF
:100010005FC0C6C65DC05CC05BC05AC059C058C096
:1000200057C056C055C080C17FC17EC17DC17CC153
:10003000D6C27AC1D4C27BC2D2C2EAC1E9C1CFC2A0
:10004000E7C1E6C1CCC2CBC2CAC299C2A8C20000F5
:1000500037343100003835320000363330040404C0
:100060000404040404020202020202030303030361
:10007000030102040810204080010204081020013E
:10008000020408102000000000000000000003042B
:100090000500000000000000000011241FBECFE595
:1000A000D4E0DEBFCDBF10E0A0E6B0E0E6EBF0E1CB
:1000B00002C005900D92A036B107D9F710E0A0E676
:1000C000B0E001C01D92AC39B107E1F765D6F2C7C7
:1000D00097CF0F931F93880F991F672B49F08C01BF
:1000E00006591F4F60E0F801808140D761E008C0E9
:1000F0008C0106591F4F61E0F801808137D760E01D
:10010000F8018081DFD61F910F9108950F931F93FF
:10011000CF93DF93EC018B0180916800909169008F
:10012000892B09F4DEC0C830D1055CF4C430D10598
:1001300094F4209709F45BC0C130D10509F04FC297
:1001400084C0CE30D10539F0C331D10541F02B97B1
:1001500009F045C21FC0B801CE01BBDF40C280918B
:10016000940090919500892B09F039C260E081E0FC
:10017000FDD661E070E080E090E04ED62FE141E0F6
:100180006CE08DE028D761E070E080E090E044D63C
:10019000202F1BC0672B31F181E090E090939500F8
:1001A0008093940060E081E0E1D661E070E080E05F
:1001B00090E032D62FE141E06CE08DE00CD761E0B9
:1001C00070E080E090E028D622ED41E06CE08DE028
:1001D00002D761E070E080E090E01ED661E081E04F
:1001E000C5D6FDC11092950010929400F8C1672BFE
:1001F00021F160E080E0BAD661E070E080E090E05C
:100200000BD62FE141E06CE08DE0E5D661E070E0D7
:1002100080E090E001D62CE841E06CE08DE0DBD698
:1002200061E070E080E090E0F7D561E080E09ED68C
:100230001092930010929200D2C1809192009091FE
:100240009300892B09F0CBC12DC0672B21F160E011
:1002500080E08CD661E070E080E090E0DDD52FE1B9
:1002600041E06CE08DE0B7D661E070E080E090E0C6
:10027000D3D522ED41E06CE08DE0ADD661E070E0D9
:1002800080E090E0C9D561E080E070D6D093930023
:10029000C0939200A4C18091920090919300019725
:1002A00009F09DC160E080E061D661E070E080E02F
:1002B00090E0B2D52FE141E06CE08DE08CD661E0BA
:1002C00070E080E090E0A8D520E041E06CE08DE0B7
:1002D00082D661E070E080E090E09ED561E080E051
:1002E0007FCF80918A0090918B00892BA9F0A091FB
:1002F0008C00B0918D00CD018F779070892B61F4C7
:100300001197B0938D00A0938C008FEF082EC6D666
:1003100010928B0010928A00FE01C431D10508F0C2
:100320005EC1ED5EFF4F099480918A0090918B0031
:10033000892B09F44DC080918E0090918F00892BFC
:1003400081F48091900090919100019751F4A091D7
:100350008C00B0918D00A130B10501F180E0082E34
:100360009DD640918C0050918D004130510581F017
:10037000012B71F0DA018AD6202D81E090E002C0D5
:10038000880F991FCA95E2F7282BDA01022E86D62C
:100390008091900090919100019749F480918E0096
:1003A00090918F00019690938F0080938E008091A2
:1003B0008E0090918F00079709F011C110928F0065
:1003C00010928E0080918C0090918D000196D2C089
:1003D000C430D10558F48091960090919700019710
:1003E00029F40115110509F0F6C0F9C0B801CE01D4
:1003F00070DE012B09F4F3C080918C0090918D0088
:10040000019709F0ECC010928D0010928C00E7C0AB
:10041000012B09F4E4C0CA30D10519F482E090E060
:1004200010C0CB30D10519F481E890E00AC0CD307E
:10043000D10519F481E091E004C02E9731F481E8F0
:1004400091E090938D0080938C0080918A00909130
:100450008B00892B09F460C0C2C0D90117D6602D6A
:1004600077276170707080E090E050DEA0918C0082
:10047000B0918D000BD6602D6695772761707070F6
:1004800081E090E043DEA0918C00B0918D00FED51C
:10049000602D6695669577276170707082E090E0B8
:1004A00035DEA0918C00B0918D00F0D5602D669561
:1004B0006695669577276170707083E090E026DE20
:1004C000A0918C00B0918D00E1D5602D62956F7088
:1004D00077276170707084E090E018DEA0918C0046
:1004E000B0918D00D3D5602D629566956695637049
:1004F00077276170707086E090E008DE80918C0054
:1005000090918D00019690938D0080938C0064E112
:1005100070E080E090E080D420918C0030918D00DC
:10052000D901B4D5802D8F3F09F097CF58C0012B4A
:1005300009F455C080918A0090918B00A0918C00A5
:10054000B0918D00892B71F0A130B10509F447C03D
:100550008FEF082EA3D510928B0010928A0081E0B5
:1005600090E008C01197D9F181E090E090938B0062
:1005700080938A0090938D0080938C0030C00C3360
:1005800011052CF461E070E082E090E017C00F3BB1
:100590001105E4F061E070E083E090E00FC00C33FF
:1005A00011052CF461E070E080E090E007C00F3BA3
:1005B000110564F061E070E081E090E08ADD81E0A7
:1005C00090E0909397008093960009C01092970056
:1005D0001092960004C0B801CE017BDD0DCFDF91F3
:1005E000CF911F910F910895BF92CF92DF92EF921A
:1005F000FF920F931F93CF93DF936C018B01B42E67
:10060000FF2441E0E42EC0E0D0E06B2D6E218C2D64
:10061000ADD4EE0C60E0802FA9D484E190E01CD42E
:1006200082E06ED4F6949695982F882797958795B3
:10063000F80E61E0802F9AD42196C830D10529F7B1
:1006400084E190E009D48F2D9927DF91CF911F91FC
:100650000F91FF90EF90DF90CF90BF900895EF92B1
:10066000FF920F931F93CF93DF9360E084E07ED4DB
:1006700041E065E070E083E090E0B6DF42E465E0F1
:1006800070E083E090E0B0DF813429F410926700DD
:10069000109266000DC0833519F481E090E004C02B
:1006A000833731F482E090E0909367008093660096
:1006B00040E065E070E083E090E096DF80916600C6
:1006C000909167001816190654F080916800909177
:1006D0006900892B21F462E0E62EF12C03C056E07C
:1006E000E52EF12CC0E0D0E000E610E00AC040E0CA
:1006F00065E070E083E090E077DFF80181938F019F
:100700002196CE15DF059CF361E084E02FD4DF91C4
:10071000CF911F910F91FF90EF900895CF93DF93AA
:100720009EDF61E080E022D461E081E01FD460912F
:100730006000603F20F08091610086FD07C081E08D
:1007400090E0909391008093900004C010929100EB
:10075000109290007727C1E0D0E06C277D27617070
:10076000707089E090E0D2DC609160007727769528
:1007700067956C277D27617070708FE090E0C6DC14
:1007800060916000772776956795769567956C27D9
:100790007D27617070708CE090E0B8DC6091600043
:1007A000772793E0769567959A95E1F76C277D27F3
:1007B0006170707088E090E0A9DC6091600077273C
:1007C00084E0769567958A95E1F76C277D276170BF
:1007D000707080E090E09ADC609160007727B5E06F
:1007E00076956795BA95E1F76C277D2761707070F3
:1007F00083E090E08BDC609160007727A6E076953F
:100800006795AA95E1F76C277D276170707081E08C
:1008100090E07CDC60E070E08091600087FD02C0C9
:1008200061E070E082E090E071DC80916600909180
:10083000670060916100019709F069C077276C2714
:100840007D27617070708BE090E060DC60916100EA
:100850007727769567956C277D27617070708AE0A1
:1008600090E054DC609161007727769567957695E6
:1008700067956C277D276170707086E090E046DC9C
:1008800060916100772753E0769567955A95E1F777
:100890006C277D276170707087E090E037DC609195
:1008A0006100772744E0769567954A95E1F76C27D4
:1008B0007D27617070708DE090E028DC60916100B0
:1008C000772735E0769567953A95E1F76C277D2790
:1008D0006170707085E090E019DC609161007727AD
:1008E00026E0769567952A95E1F76C277D2761705C
:1008F000707084E090E00ADC60E070E0809161005C
:1009000087FD02C061E070E08EE090E068C077276C
:100910006C277D27617070708BE090E0F7DB609151
:1009200061007727769567956C277D2761707070D9
:100930008EE090E0EBDB609161007727769567951C
:10094000769567956C277D27617070708AE090E0DE
:10095000DDDB609161007727B3E076956795BA9506
:10096000E1F76C277D27617070708DE090E0CEDB41
:10097000609161007727A4E076956795AA95E1F7E5
:100980006C277D276170707087E090E0BFDB60911D
:1009900061007727F5E076956795FA95E1F76C2782
:1009A0007D276170707085E090E0B0DB6091610040
:1009B0007727E6E076956795EA95E1F76C277D273E
:1009C0006170707084E090E0A1DB60E070E0809185
:1009D000610087FD02C061E070E086E090E096DB98
:1009E00080916600909167001816190634F0809186
:1009F000680090916900892BC1F0609162007727AF
:100A000080E190E083DB60916300772781E190E0F3
:100A10007DDB60916400772782E190E077DB609175
:100A20006500772783E190E071DBDF91CF91089536
:100A300060E084E09BD241E065E070E083E090E01C
:100A4000D3DD43E465E070E083E090E0CDDD40E09D
:100A500065E070E083E090E0C7DD41E065E070E0D4
:100A600083E090E0C1DD40E065E070E083E090E08D
:100A7000BBDD61E084E07AD264E670E080E090E083
:100A8000CBD160E084E072D241E065E070E083E0C9
:100A900090E0AADD44E465E070E083E090E0A4DD4E
:100AA00040E065E070E083E090E09EDD41E065E0DD
:100AB00070E083E090E098DD40E065E070E083E086
:100AC00090E092DD40E065E070E083E090E08CDD56
:100AD00040E065E070E083E090E086DD40E065E0C6
:100AE00070E083E090E080DD40E065E070E083E06E
:100AF00090E07ADD61E084E039D264E670E080E085
:100B000090E08AD160E084E031D241E065E070E0BD
:100B100083E090E069DD43E465E070E083E090E02D
:100B200063DD40E065E070E083E090E05DDD40E0A3
:100B300065E070E083E090E057DD40E065E070E064
:100B400083E090E051DD40E065E070E083E090E01C
:100B50004BDD40E065E070E083E090E045DD40E0A3
:100B600065E070E083E090E03FDD40E065E070E04C
:100B700083E090E039DD61E084E0F8D10895CF931F
:100B8000DF931092970010929600109295001092A9
:100B9000940060E082E096D161E083E093D161E06F
:100BA00084E090D161E085E08DD160E086E08AD17B
:100BB00060E087E087D160E088E084D160E089E090
:100BC00081D160E08AE07ED160E08BE07BD160E0A3
:100BD00083E178D161E080E075D161E081E072D19C
:100BE00061E08CE06FD161E08DE06CD161E084E088
:100BF000BDD161E085E0BAD161E083E0B7D181E0A9
:100C000090E09093690080936800C0E0D0E027DD19
:100C10002196C530D105D9F7C0E0D0E020DD809124
:100C2000680090916900892B11F490E005C090E074
:100C30008091600087FF91E0892F99279093690048
:100C4000809368002196C431D10541F7EAE6F0E0CF
:100C50002FEF3FEF2193319340E0EA38F407D1F7CB
:100C6000892B01F187E090E09093870080938600C4
:100C700088E090E0909375008093740089E090E0A4
:100C800090937900809378008AE090E090937300CD
:100C9000809372008BE090E09093770080937600D1
:100CA000C7DE43C087E090E090936B0080936A00BA
:100CB00088E090E090936D0080936C0089E090E074
:100CC00090936F0080936E008AE090E090937100A3
:100CD000809370008BE090E090937300809372009B
:100CE00083E190E0909377008093760060E081E06C
:100CF0003DD161E070E080E090E08ED02FE141E0F6
:100D00006CE08DE068D161E070E080E090E084D03C
:100D10002FEF41E06CE08DE05ED161E070E080E0BB
:100D200090E07AD061E081E021D110928B001092A6
:100D30008A0010928F0010928E002FE730E0D901C8
:100D4000A5D1802D8F3F21F08FEFD901082EA6D19C
:100D50002FEF30E0D9019AD1802D8F3F21F08FEF16
:100D6000D901082E9BD12FE731E0D9018FD1802DF9
:100D70008F3F21F08FEFD901082E90D12FEF31E076
:100D8000D90184D1802D8F3F21F08FEFD901082E1A
:100D900085D1DF91CF9108956CD0F1DEBFDCFECF1D
:100DA0001F920F920FB60F9211248F939F93AF93C0
:100DB000BF938091980090919900A0919A00B09172
:100DC0009B000196A11DB11D8093980090939900FE
:100DD000A0939A00B0939B00BF91AF919F918F9188
:100DE0000F900FBE0F901F90189560919800709112
:100DF000990080919A0090919B0027E0660F771FE1
:100E0000881F991F2A95D1F72DE730E040E050E088
:100E10001BD1CA01B9010895AF92BF92CF92DF9260
:100E2000EF92FF920F931F935B016C01DEDF7B015A
:100E30008C01DBDF6E197F09800B910B6A157B0536
:100E40008C059D05B0F31F910F91FF90EF90DF90FF
:100E5000CF90BF90AF900895019751F0880F991FE0
:100E6000880F991F02972FB7F8940197F1F72FBFBA
:100E700008957894109298001092990010929A0018
:100E800010929B0083B7826083BF83B7816083BF6A
:100E900089B7816089BF8EB582608EBD8EB5816055
:100EA0008EBD8FB581608FBD85B5846085BD85B5EC
:100EB000806485BD3F983E9A329A319A309A379A2B
:100EC0001AB80895282F3327C9018F589F4FFC0166
:100ED0009491235A3F4FF9018491882381F0E82FA0
:100EE000FF27E25BFF4FE491FF27662329F480810F
:100EF00090958923808308958081892B808308952C
:100F0000482F5527CA018B579F4FFC012491CA01D6
:100F10008F589F4FFC019491435A5F4FFA013491CF
:100F2000332319F480E090E00895222381F02330E8
:100F300019F48FB58F7704C0243021F48FB58F7DDD
:100F40008FBD05C0253019F485B58F7D85BDE32F94
:100F5000FF27E85AFF4FE491FF27808120E030E02F
:100F6000892311F021E030E0C9010895482F552769
:100F7000CA018B579F4FFC012491CA018F589F4F84
:100F8000FC019491435A5F4FFA013491332311F1DC
:100F9000222381F0233019F48FB58F7704C02430D9
:100FA00021F48FB58F7D8FBD05C0253019F485B52F
:100FB0008F7D85BDE32FFF27ED5AFF4FE491FF277B
:100FC000662329F480819095892380830895808108
:100FD000892B80830895CF92DF92EF92FF920F9337
:100FE0001F93CF93DF93E82EF62EC42ED22EC0E0AF
:100FF000D0E007E010E06D2D7727CC2039F40C2EDF
:1010000002C0759567950A94E2F706C0002E02C0EB
:10101000759567950A94E2F761708E2DA7DF61E000
:101020008F2DA4DF60E08F2DA1DF219601501040AD
:10103000C830D10501F7DF91CF911F910F91FF903B
:10104000EF90DF90CF900895A1E21A2EAA1BBB1B50
:10105000FD010DC0AA1FBB1FEE1FFF1FA217B30784
:10106000E407F50720F0A21BB30BE40BF50B661F9A
:10107000771F881F991F1A9469F76095709580955E
:1010800090959B01AC01BD01CF010895E199FECF80
:10109000BFBBAEBBE09A11960DB20895E199FECFA9
:1010A000BFBBAEBB0DBA11960FB6F894E29AE19AA7
:0610B0000FBE0895FFCF02
:00000001FF
